:0E0000000C94DD000C94C4010C94AC020C9422
:10000E000C010C9400000C9400000C9400000C9455
:10001E0000000C9400000C94E7020C9400000C9469
:10002E0000000C9400000C94A8040C9400000C9496
:10003E0000000C9400000C9400000C94CA020C9466
:10004E0000000C9400000C9400000C9400000C9422
:10005E0000000C9400000C9400001027E8036400CC
:10006E000A00010000100001100001000000010054
:10007E00000102040810200000030602050104001E
:10008E00060402070005030107060007060007061F
:10009E00000507060007060007060004070600070E
:1000AE000600070600030706000706000706000203
:1000BE000029CD007B52A400007B2952CDA400CD97
:1000CE007BA429005200E0005500AA0000070D1481
:1000DE001A20272D343A40474D53595F656B71777F
:1000EE007D82888D93989DA2A7ACB1B5BABEC3C7C9
:1000FE00CBCFD2D6DADDE0E3E6E9EBEEF0F2F4F6C2
:10010E00F8F9FAFBFCFDFEFEFFFFFFFFFEFEFDFC15
:10011E00FBFAF9F8F6F4F2F0EEEBE9E6E3E0DD00D7
:10012E0010272701A4011300640000000000000046
:10013E0000000000000000000000000000000000B1
:10014E0000000000010002007A00010006007C00A1
:10015E00070000037E0007000A0386000800120352
:10016E008E0028001E03960007004703BE000600FF
:10017E004F03C60007005703CC0001006503D400EF
:10018E0001009103D60001009203D8005300EF0442
:10019E00DA00020046052E0102004A053001020077
:1001AE004C0532010100A00534010000F894EE2741
:1001BE00EFBBF1E0F5BFE5BF8DE0A2E0BB27ED930D
:1001CE008A95E9F780E098E0A0E0B1E0ED93019721
:1001DE00E9F7E2E5F1E085919591009761F0A5913F
:1001EE00B59105901590BF01F00105900D92019704
:1001FE00E1F7FB01F0CFE0E0EEBBEFEFEDBFE8E0A3
:10020E00EEBFC0E0D3E00C94E0080A92AA93EA9302
:10021E00FA93EFB7EA93E0916D03E03011F00C948E
:10022E002C01A0E04A99A1E0EA2FEE0FEE0F0E2E60
:10023E00A0E01D99A1E0EA2FEE0FA02DAE0FE0E099
:10024E001C99E1E0EA0FE0937503A0916D03A130D4
:10025E0011F00C944601A0E04A9BA1E0EA2FEE0FAC
:10026E00EE0F0E2EA0E01D9BA1E0EA2FEE0FA02DAB
:10027E00AE0FE0E01C9BE1E0EA0FE0937503A09166
:10028E006E03A13011F00C945401E0917503F0E06F
:10029E00EE5EFC4FE081E0937503E0917503F0E0B4
:1002AE00E65FFC4FE081A0917403EA1711F00C9405
:1002BE00A301E0917503E0937403A0916103AA304A
:1002CE0010F40C947101E0916103E0936003689463
:1002DE0026F803C0E0E0E0936003E0E0E0937703EC
:1002EE00E0917403F0E0E95BFC4FE081A0915905C9
:1002FE00EA0FE0939003E0917403F0E0E15BFC4FB2
:10030E00E081EA0FE0939103E0917403F0E0E95A83
:10031E00FC4FE081EA0FE0939203E0917403F0E06A
:10032E00E050FD4FE0814E2AE0917403F0E0E05082
:10033E00FD4FE0813E2A0FC0A0917803E0E00E94BD
:10034E0029230E2EE3E00E942923E02911F40C94B8
:10035E00B201689421F8E0917403A0917503EA1735
:10036E0011F00C94BD01E0E0E0937103E991EFBF51
:10037E00F991E991A991099018950A921A92AA9366
:10038E00EA93FA93EFB7EA93E0916D03E03011F040
:10039E000C94E501A0E04A99A1E0EA2FEE0FEE0FD2
:1003AE000E2EA0E01D99A1E0EA2FEE0FA02DAE0FAC
:1003BE00E0E01C99E1E0EA0FE0937503A0916D0374
:1003CE00A13011F00C94FF01A0E04A9BA1E0EA2FAE
:1003DE00EE0FEE0F0E2EA0E01D9BA1E0EA2FEE0F0A
:1003EE00A02DAE0FE0E01C9BE1E0EA0FE093750359
:1003FE00A0916E03A13011F00C940D02E0917503E3
:10040E00F0E0EE5EFC4FE081E0937503E091750342
:10041E00F0E0E65FFC4FE081A0917403EA1711F063
:10042E000C945B02E0917503E0937403A091610359
:10043E00AA3010F40C942A02E0916103E093600359
:10044E00689426F803C0E0E0E0936003E0E0E093F8
:10045E007703E0917403F0E0E95BFC4FE081A0913B
:10046E005905EA0FE0939003E0917403F0E0E15B2D
:10047E00FC4FE081EA0FE0939103E0917403F0E00A
:10048E00E95AFC4FE081EA0FE0939203E091740386
:10049E00F0E0E050FD4FE0814E2AE0917403F0E071
:1004AE00E050FD4FE0813E2AE0917403A091750368
:1004BE00EA1711F00C946602E0E0E0937103A32DAD
:1004CE00EFE30E9429230E2EA0E04A99A1E0E0E07E
:1004DE000E942923E0211E2EA0E021FCA1E0E1E0F4
:1004EE000E9429230E2EA0E04A99A1E0E0E00E948E
:1004FE002923E021E12911F40C94A402E89421F8B7
:10050E003324E0914605F0914705E0934805F093BA
:10051E004905E0E0E0934605E0934705E0916E0360
:10052E00E03011F40C94A002E8941D9B689423F81B
:10053E0004C0E8941D99689423F8E991EFBFF991EE
:10054E00E991A991199009901895EA93E0E0E0934A
:10055E00E403E093E303E093E203E093E103E0932B
:10056E00E003E093DF03E0937A03399A209A579AD7
:10057E00419828985F98E1E0E4BDE093B000F09ACE
:10058E00F49AE9911895EA93FA93EFB7EA931A93CE
:10059E001091C600E091C000EC7111F00C94E102D4
:1005AE00E091CA05EF5FE093CA05E150F0E0EE5529
:1005BE00FA4F10831991E991EFBFF991E9911895CE
:1005CE000A921A92AA93BA93EA93FA93EFB7EA931E
:1005DE00E0915405F0915505A0915205B091530547
:1005EE00EA0FFB1FE0935205F0935305E09153057C
:1005FE00E07E11F40C946203E0E0E0938F03E0914F
:10060E005305E07811F40C941103E0918F03E4602C
:10061E00E0938F03E0915305E07411F40C941C03E6
:10062E00E0918F03E260E0938F03E0915305E07257
:10063E0011F40C942703E0918F03E160E0938F0394
:10064E00E0915305EF71E0935305E0918F03A09174
:10065E009003EA0FE0939003E0918F03A091910332
:10066E00EA0FE0939103E0918F03A0919203EA0FBA
:10067E00E0939203A0919003A63F10F40C944C03C8
:10068E00E0919003E65FE0939003A0919103A63F63
:10069E0010F40C945703E0919103E65FE0939103FD
:1006AE00A0919203A63F10F40C946203E091920382
:1006BE00E65FE0939203992011F40C94AE03E0915F
:1006CE009003F0E0E251FC4FE081A0917A03AE1767
:1006DE0010F00C947703E0917A03E093B30008C016
:1006EE00E0919003F0E0E251FC4FE081E093B30023
:1006FE00E0919103F0E0E251FC4FE081A0917A038A
:10070E00AE1710F00C948F03E0917A03E7BD07C08B
:10071E00E0919103F0E0E251FC4FE081E7BDE09102
:10072E009203F0E0E251FC4FE081A0917A03AE1704
:10073E0010F00C94A603E0917A03E8BD07C0E09197
:10074E009203F0E0E251FC4FE081E8BD47C0E0913A
:10075E005F03F0E0ED56FC4FE081A0917B03AE17F6
:10076E0010F00C94BF03E0917B03E093B30008C03C
:10077E00E0915F03F0E0ED56FC4FE081E093B300B3
:10078E00E0915F03F0E0E455FC4FE081A0917B0324
:10079E00AE1710F00C94D703E0917B03E7BD07C0B2
:1007AE00E0915F03F0E0E455FC4FE081E7BDE0919E
:1007BE005F03F0E0EB53FC4FE081A0917B03AE179B
:1007CE0010F00C94EE03E0917B03E8BD07C0E091BE
:1007DE005F03F0E0EB53FC4FE081E8BDA0914605CE
:1007EE00B0914705A031E7E2BE0710F00C94080463
:1007FE00E0914605F09147053196E0934605F0935A
:10080E004705A0916003E0E00E943D230E2EA091CB
:10081E008103E8E00E943823E02111F40C94510486
:10082E00E0917403E85FE0935F03E0918103EF5F73
:10083E00E093810326FE07C0E89426F8E091740346
:10084E00E0935F0326C0A0918003BB27E091600375
:10085E00F0E0AE0FBF1F599714F40C944304EEEF63
:10086E00E0937B03A0918003E9E1EA1BA091600372
:10087E00AE1BA09360030DC0E0916003AAE0EA02F4
:10088E00F001A0917A03EA0FE0937B03E0E0E0939E
:10089E0060030DC0E0917403E0935F03E0917A036F
:1008AE00E0937B03E0E0E0938103E0936003A0918B
:1008BE006003A13010F40C946D04E0917403F0E029
:1008CE00EA51FC4FE081E093620308C0E0917403AB
:1008DE00F0E0E252FC4FE081E0936203E0916203AC
:1008EE00E17011F4399801C0399AE0916203E27017
:1008FE0011F4209801C0209AE0916203E47011F483
:10090E00579801C0579AE0916203E87011F441982C
:10091E0001C0419AE0916203E07111F4289801C080
:10092E00289AE0916203E07211F45F9801C05F9A19
:10093E00E991EFBFF991E991B991A99119900990B7
:10094E0018950A921A926A937A938A939A93AA9313
:10095E00BA93EA93FA93EFB7EA937894E0917F0310
:10096E00EF5FE0937F03A0917F03A83010F40C9407
:10097E00C804E0E0E0937F03E0917E03EF5FE09335
:10098E007E03A0916C03A23010F40C94D304E0917A
:10099E006C03E150E0936C03E0917703EF5FE0931B
:1009AE007703A0917703AD3310F40C945105E4E175
:1009BE00E0937703E0916D03E03011F00C94FB04AB
:1009CE00A0E04A99A1E0EA2FEE0FEE0F0E2EA0E066
:1009DE001D99A1E0EA2FEE0FA02DAE0FE0E01C99BD
:1009EE00E1E0EA0FE0937603A0916D03A13011F0E0
:1009FE000C941505A0E04A9BA1E0EA2FEE0FEE0F36
:100A0E000E2EA0E01D9BA1E0EA2FEE0FA02DAE0F43
:100A1E00E0E01C9BE1E0EA0FE0937603A0916E0309
:100A2E00A13011F00C942605E0917603F0E0EE5E15
:100A3E00FC4FE081E0937503E093740306C0E091F0
:100A4E007603E0937503E0937403E0917403F0E092
:100A5E00E95BFC4FE081EC5EA0915905EA0FE09353
:100A6E009003E0917403F0E0E15BFC4FE081EC5EFB
:100A7E00EA0FE0939103E0917403F0E0E95AFC4F22
:100A8E00E081EC5EEA0FE0939203E0E0E093540520
:100A9E00E0935505E0917503A09174030E942E23F7
:100AAE000E2EA0918405B0918505E4E6F0E00E943B
:100ABE0060230E22A0911A03E0E00E942923E02178
:100ACE001E2EE0917503A09174030E942E230E2E0C
:100ADE00A0918405B0918505ECE9FFEF0E945A23A1
:100AEE000E22A0911A03E1E00E942923E021E129C0
:100AFE000E2EA0917403E0E00E9429230E2AE7E057
:100B0E000E942923E02911F40C94E805E091710369
:100B1E00EF5FE0937103A0917103A63010F40C9473
:100B2E00E805E0E0E0937A03E0939B03E0939A03F9
:100B3E00E0939903E0939803E0939703E093960371
:100B4E00E0939503E0939403E0939303E093B4034F
:100B5E00E093B303E093B203E093B103E093B003E9
:100B6E00E093AF03E093AE03E093AD03E093AC03E9
:100B7E00E093CD03E093CC03E093CB03E093CA0361
:100B8E00E093C903E093C803E093C703E093C60361
:100B9E00E093C503E093E603E093E503E093E403FB
:100BAE00E093E303E093E203E093E103E093E003D9
:100BBE00E093DF03E093DE034424F39AE5E0E09351
:100BCE007103E0E0E0937A00E0914603F0E0E25E2C
:100BDE00FC4FE081E0931D03A2E7B5E0F0E0EE0FDD
:100BEE00FF1FAE0FBF1FE0917800F0917900ED93DB
:100BFE00FC93E0914603EF5FE0934603A09146031A
:100C0E00A83210F40C940E06E0E0E0934603E09157
:100C1E004603F0E0E25EFC4FE081E05CE0937C0096
:100C2E0084E08A95F1F7E6ECE0937A00A0911D033B
:100C3E00A73011F00C94DC06E0918005F09181054F
:100C4E00A0918805B0918905EA1BFB0BE0935E0528
:100C5E00F0935F05E0918005F0918105A0915C0510
:100C6E00B0915D05EA1BFB0BE0936C05F0936D05EF
:100C7E00A0915E05B0915F05EFEFFFEF0E9460233C
:100C8E000E2EA0917A03E0E00E943D23E02111F4A4
:100C9E000C94560625FE03C0E1E0E0936403A09198
:100CAE005E05B0915F05E4E1F0E00E9460230E2E38
:100CBE00A0917A03E1E00E943D230E22A091090348
:100CCE00E0E00E942923E02111F40C948A06E091C1
:100CDE007A03E150E0937A03A0915E05B0915F052F
:100CEE00E2E3F0E00E9460230E2EA0917A03E3E08F
:100CFE000E943D23E02111F40C948A06E0917A03C0
:100D0E00E350E0937A03E0918C05F0918D056091AC
:100D1E008E0570918F050E940123A0916C05B091F4
:100D2E006D050E9424230E9472230E2EA0917A0339
:100D3E00E0E00E943D230E22A0910903E0E00E9414
:100D4E002923E0211E2EA0916C05B0916D051A96F7
:100D5E00E0918C05F0918D0560918E0570918F0557
:100D6E000E9401230E9424230E9472230E2EA09122
:100D7E007A03E0E00E943D230E22A0910903E1E0F8
:100D8E000E942923E021E12911F40C94DC06E09164
:100D9E007A03E150E0937A03E0910903E03011F019
:100DAE000C94DC06E1E0E0936403E0911D03E03077
:100DBE0011F00C945607A0918903B0918A03E0912B
:100DCE007205F0917305EA1BFB0BE0936405F0933B
:100DDE006505E0916205F0916305A0917205B091F1
:100DEE007305EA17FB0714F00C940C07A09162052B
:100DFE00B0916305E0917205F0917305EA1BFB0B50
:100E0E00E0936005F093610505C0E0E0E0936005B6
:100E1E00E0936105A0916405B0916505EFEFFFEFDA
:100E2E000E9460230E2EA0917A03E0E00E943D23E3
:100E3E00E02111F40C94280725FE03C0E1E0E093B5
:100E4E006403A0916405B0916505E8E2F0E00E94AC
:100E5E0060230E2EA0917A03E1E00E943D23E02153
:100E6E0011F40C945607E0917A03E150E0937A0363
:100E7E00A0916405B0916505E0E5F0E00E94602365
:100E8E000E2EA0917A03E3E00E943D23E02111F49F
:100E9E000C945607E0917A03E350E0937A03A09105
:100EAE001D03A63011F00C94D308A0917E05B091CD
:100EBE007F05E0914A05F0914B053196AE17BF07BD
:100ECE0010F00C948607A0916805B0916905E0E0DA
:100EDE00F0E00E9460230E2EA0918205B091830552
:100EEE00E0E0F0E00E9442230E22A0910903E0E030
:100EFE000E942923E02111F40C94860701C005C03D
:100F0E0025FE03C0E1E0E0936403A0917E05B0915D
:100F1E007F051196E0914A05F0914B05AE17BF077C
:100F2E0010F00C94B607A0916805B0916905E0E049
:100F3E00F0E00E9460230E2EA0918205B0918305F1
:100F4E00E0E0F0E00E9442230E22A0910903E0E0CF
:100F5E000E942923E02111F40C94B60701C03AC077
:100F6E00A0917E05B0917F051396E0914A05F09110
:100F7E004B050E9466230E2EA0917A03E5E00E9497
:100F8E003D230E22A0916C05B0916D05E5E0F0E0D9
:100F9E000E946023E02111F40C94DA07E0917A03A9
:100FAE00E550E0937A03A0917A03E0E00E943D239E
:100FBE000E2EA0916C05B0916D05E5E0F0E00E945B
:100FCE006023E02111F40C94F107E0917A03E150D3
:100FDE00E0937A03A0916805B0916905E0E0F0E036
:100FEE000E9442230E2EA0918205B0918305E0E06F
:100FFE00F0E00E9460230E22A0910903E0E00E941F
:10100E002923E02111F40C94B308A0917E05B09130
:10101E007F05E0914C05F0914D05EA17FB0710F0A6
:10102E000C944108E1E0E0936403A0917A03A130AF
:10103E0010F40C942708E0917A03E150E0937A03C0
:10104E00A0917E05B0917F05E0914C05F0914D0584
:10105E003A960E946C230E2EA0917A03E5E00E9430
:10106E003D23E02111F40C944108E0917A03E55000
:10107E00E0937A03A0917E05B0917F05E0914C0537
:10108E00F0914D050E9466230E2EE0918C05F09195
:10109E008D0560918E0570918F050E940123A091A0
:1010AE006C05B0916D050E9424230E947A23E021E5
:1010BE0011F40C94B308E0917A03A0918205B091DB
:1010CE008305F0E0EA17FB0714F00C947308E09127
:1010DE007A03EF5FE0937A03E0917A03A0918205A1
:1010EE00B0918305F0E0AE17BF0714F00C9484089E
:1010FE00E0917A03E150E0937A03A0917E05B091DE
:10110E007F051A96E0914C05F0914D050E946623DD
:10111E000E2EE091A105F0E0A5EFB0E0AE1BBF0BE7
:10112E00E0917A03F0E00E9460230E2AE0917A03A8
:10113E00F0E0A0918205B0918305AE1BBF0BE5E0F8
:10114E00F0E00E946023E02111F40C94B308E091CA
:10115E007A03EE5FE0937A03A0910903E1E00E9427
:10116E0029230E2EA0917E05B0917F05E0914C05AE
:10117E00F0914D0535960E946C230E22A0917A03B4
:10118E00E5E00E943D23E02111F40C94D308E09198
:10119E007A03E550E0937A03E991EFBFF991E99173
:1011AE00B991A99199918991799169911990099023
:1011BE0018956F978CE1A0E0B0E0E6E3F1E00E94B5
:1011CE00502414E0E0E8E0936100E0E0E093610079
:1011DE00EFE0E4B9E0E3E5B9E2E0E7B9E0E0E8B971
:1011EE00E0EFEAB9ECE0EBB9E1EAE4BDE1E0E5BD40
:1011FE00E0E0E6BDE7BDE8BDE1EAE0938000E2E0B5
:10120E00E0938100E0E0E0938500E0938400E093BA
:10121E008700E0938600E0938900E0938800E093D6
:10122E008B00E0938A00E093B600E1E8E093B00013
:10123E00E1E0E093B100E0E0E093B200E093B300B0
:10124E00E093B400E0936E00E1E0E0936F00E09372
:10125E007000EDE0E0936900E3E0EDBBECBBE1E094
:10126E00E0936800E0E3E0936B00E1E0EBBBE0E0CD
:10127E00E093C000E0E9E093C100E6E0E093C20035
:10128E00E0E0E093C500ECE0E093C400E0E4E0931E
:10129E007C00E0E8E0BFE0E0E0937F00ECBDE0938F
:1012AE00BC00E093B200E6BD419828985F98ACE28E
:1012BE00B1E00E9446213998209A5798E4E6E093CF
:1012CE00B300E7BDE0E0E8BD84E68A95F1F7E09370
:1012DE00B300E7BDE8BD8CE291E00197F1F73998D4
:1012EE002098579AE093B300E4E6E7BDE8BD84E6A4
:1012FE008A95F1F7E0E0E093B300E7BDE8BD8CE23C
:10130E0091E00197F1F7399A20985798E4E6E09327
:10131E00B300E0E0E7BDE4E6E8BD88E78A95F1F7C3
:10132E00E0E0E093B300E7BDE8BDA2E3B0E00E94C9
:10133E004621E7E4E0937C0088E28A95F1F7E6EC3B
:10134E00E0937A00A1E0B0E00E944621E09178009F
:10135E00F0917900E0935C05F0935D05E0E0E09399
:10136E007A00A1E0B0E00E944621E0E4E0937C0028
:10137E0088E28A95F1F7E6ECE0937A00A1E0B0E01E
:10138E000E944621E0917800F0917900E093620589
:10139E00F0936305E0E0E0937A00E1E0E0937703F9
:1013AE00F798A0915C05B0915D05EAEFF0E00E9420
:1013BE0060230E2EE6E9F0E00E945A23E02911F494
:1013CE000C94F109E8ECF0E0E0935C05F0935D0518
:1013DE00F19A01C0F198A0916205B0916305E2E81F
:1013EE00F0E00E9460230E2EEAE5F0E00E945A2300
:1013FE00E02911F40C940B0AE0E7F0E0E0936205AB
:10140E00F0936305F29A01C0F2987894A091850347
:10141E00B0918603AC32E1E0BE0710F00C94450AA1
:10142E00E0918503F09186033196E0938503F09366
:10143E008603A0918503B0918603AC32E1E0BE072E
:10144E0011F00C94450A6624E0E0EF8BAF89A031D1
:10145E0010F00C943C0AEF89F0E0EE55FA4FA0E044
:10146E00A083EF89EF5FEF8BF1CFE7E9F0E0E09338
:10147E008503F0938603E0E0E093CA05A091A205F0
:10148E00EAE60E9429230E2EA091A305EFE00E940A
:10149E0029230E22A091CA05E0E10E942923E02112
:1014AE0011F40C94590CE1E0EF8BAF89AF3010F0D2
:1014BE000C946F0AEF89F0E0EE55FA4FE081A0919F
:1014CE006703EA0FE0936703EF89EF5FEF8BEDCFD2
:1014DE00E091B105A0916703EA1711F00C94430C4B
:1014EE00E0E0E0938503E0938603EEE1E0936C0386
:1014FE00E091A405EF701E2FA0E0B0E00E94292419
:10150E00EC5FA091A4050E940923E170ED8FAD8DD3
:10151E00A13011F00C94BA0AE091A505E370E093A6
:10152E006A03A5EAB5E0EC91E695E695EC93E091B9
:10153E00A505E3702E2FA5EAB5E0EC91E695E695AC
:10154E00EC93E091A505E3703E2FA5EAB5E0EC9192
:10155E00E695E695EC93E091A505E3700E2F50907D
:10156E00A6058090A705A0E0B0E00E942924EC5FBC
:10157E00A091A8050E940923E170E0936303E09116
:10158E00AF05E170EC8FA0916303A13011F00C94C4
:10159E00670BA0E0B0E00E942924F0E0E755FA4F77
:1015AE00A081A93C10F40C94EB0AEFEFF0E0E0936D
:1015BE006805F0936905E0918805F0918905E0933F
:1015CE006A05F0936B054CC0A0E0B0E00E942924A0
:1015DE00F0E0E755FA4FE081F0E00E941F230E94F1
:1015EE00B621AAE0B7ED83EA9FE30E944022A8E667
:1015FE00B5E00E947F21ED93FC93E0915C05F091A4
:10160E005D05A0918805B091890580918A0590911C
:10161E008B050E941F230E941C240E94F8227F9398
:10162E006F93FF93EF93A0E0B0E00E942924F0E0C7
:10163E00E755FA4FE081F0E0AF91BF918F919F9106
:10164E000E941F230E94AF23DF01CB01E8ECF0E0E4
:10165E0060E070E00E94F123E0936A05F0936B0561
:10166E00E0E0E0938205E0938305AC8DE1E00E941B
:10167E0029230E2EA0916903E3E00E943823E02176
:10168E0011F40C945F0BE0917D03E03011F00C949B
:10169E00540BE0917A03E0937D03E0917D03F0E03B
:1016AE00E0936805F0936905E0E0E093680307C0F6
:1016BE00E0E0E0937D03E0916903E093680379C075
:1016CE00EB8DE03011F00C94B30BA0E0B0E00E9473
:1016DE002924F0E0E755FA4FE081F0E00E941F2345
:1016EE000E94B621AAE0B7ED83EA9FE30E94402252
:1016FE00ADE8B3E00E947D21ED93FC93A0918D03A4
:10170E00B0918E03EFEFF0E0EA1BFB0B0F01EFEF52
:10171E00F0E0EA1BFB0BD0010E948223DF01EFEF0A
:10172E00F0E00E94B4230F01A0918D03B0918E03BF
:10173E00EFEFF0E0EA1BFB0BD0010E948223DF01EA
:10174E00EFEFF0E00E94B423AFEFB0E0AE1BBF0BA3
:10175E00A0938205B0938305AB8DA13011F00C944C
:10176E00D70BA0E0B0E00E942924F0E0E755FA4F35
:10177E00E081F0E0E0938D03F0938E03E091A105FC
:10178E00F0E0A0918D03B0918E030E948223DF01C1
:10179E00E8ECF0E00E94B423E0938D03F0938E0307
:1017AE00E0E0E0936805E0936905E0936A05E09355
:1017BE006B05A0910903A13011F00C94F50BE0E03C
:1017CE00E0936805E0936905E0936A05E0936B0585
:1017DE00EFEFF0E0E0938205F0938305A0E0B0E038
:1017EE000E942924A091A8050E940923E170E0938C
:1017FE001A03A0916903E3E00E9429230E2EA09103
:10180E006805B0916905E0E0F0E00E9460230E22C9
:10181E00AC8DE1E00E9429230E22A0916503E0EE3B
:10182E000E942923E02111F40C94210CE09154051F
:10183E00E0936503EC8DE03011F00C94290CE0EE92
:10184E00E0936503AFEAB5E0EC91E695EC93E09199
:10185E00AF05E0FB24F8AFEAB5E0EC91E695E6952E
:10186E00E695EC93E091AF05EF70E98FE091B0054E
:10187E00E0935605E1E06E2EE0E0EF8BAF89A031EC
:10188E0010F00C94540CEF89F0E0EE55FA4FA0E0F6
:10189E00A083EF89EF5FEF8BF1CFE0E0E093CA0515
:1018AE00E0936703A0916303E0E00E9429230E2ECC
:1018BE00AB8DE1E00E9429230E22A0918503B09109
:1018CE008603E6E9F0E00E9466230E22A0E020FCEB
:1018DE00A1E0E0E00E942923E02111F40C949A0C7F
:1018EE00E091A105F0E0AFEFB0E00E942224EA1BE8
:1018FE00FB0BA0918D03B0918E03EA0FFB1FE093BB
:10190E008205F0938305A0918205B0918305A030E6
:10191E00E1E0BE0714F40C949A0CEFEFF0E0E093C4
:10192E008205F0938305A091A205EAE60E94292381
:10193E000E2EA091A305EFE00E9429230E22A09166
:10194E00CA05E0E10E943D23E02111F40C94BB0C8A
:10195E00E0914E05F0914F053196E0934E05F093D0
:10196E004F05E0E0E093CA05A091A205ECE60E94C7
:10197E0029230E2EA091A305EFE00E9429230E220B
:10198E00A091CA05E0E10E942923E02111F40C94F4
:10199E00E70EE1E0EF8BAF89AF3010F00C94E50C61
:1019AE00EF89F0E0EE55FA4FE081A0916703EA0F60
:1019BE00E0936703EF89EF5FEF8BEDCFE091B10519
:1019CE00A0916703EA1711F00C94D10EE0E0E093BA
:1019DE008503E09386035091A405E091A605E3707C
:1019EE004E2FA6EAB5E0EC91E695E695EC93E091E4
:1019FE00A605E170EE8FA6EAB5E0EC91E695EC93C4
:101A0E00AE8DA13011F00C94110DE42FA0E0B0E0DA
:101A1E000E943524A0E0B0E00E942924E41711F0C2
:101A2E000C94CF0EE091A505E170AE2EA5EAB5E0BF
:101A3E00EC91E695EC93E091A505E170E0936D03D2
:101A4E00A5EAB5E0EC91E695EC93E091A505E17081
:101A5E00E0936E03A5EAB5E0EC91E695EC93E09188
:101A6E00A505E170EB8FA5EAB5E0EC91E695EC9358
:101A7E00E091A505E370E0936903A5EAB5E0EC916A
:101A8E00E695E695EC93E091A505E170EA8FA5EA5F
:101A9E00B5E0EC91E695EC93E091A505E0FB27F817
:101AAE00E091A605E170EA8BA6EAB5E0EC91E69529
:101ABE00EC93E091A605E170E88FA6EAB5E0EC9113
:101ACE00E695EC93E091A605E170EE8BA6EAB5E003
:101ADE00EC91E695EC93E091A605E093EE04E0918F
:101AEE00A705FF2766277727E0938805F0938905DA
:101AFE0060938A0570938B05A0918805B091890536
:101B0E0080918A0590918B050E944A2414F00C94C2
:101B1E00930D689425F802C0E89425F8E0918805A5
:101B2E00F091890560918A0570918B050E94B6210E
:101B3E00DF01CB01EAE8FEE864E67DE30E948E2237
:101B4E00A8E8B5E00E947F210E941724E0915C0571
:101B5E00F0915D05A0918805B091890580918A0567
:101B6E0090918B050E941F230E94F322E09388051B
:101B7E00F093890560938A0570938B05A091880573
:101B8E00B091890580918A0590918B05A030E4E093
:101B9E00BE07E0E08E07E0E09E0714F40C94E30D20
:101BAE00EFEFF3E060E070E0E0938805F0938905D5
:101BBE0060938A0570938B05E091A805FF27662731
:101BCE007727E0938C05F0938D0560938E057093C7
:101BDE008F050E94B621DF01CB01EAE8FEE864E63C
:101BEE007DE30E948E22ACE8B5E00E947F210E9428
:101BFE001724E091A905ED8BAD89EAE0EA9FF0018B
:101C0E00DF01E091AA05F0E0AE1BBF0BA0934A05E1
:101C1E00B0934B05AD89EAE0EA9FF001DF01E09158
:101C2E00AB05F0E0EA0FFB1FE0934C05F0934D057A
:101C3E00E091AC05F0E0E0938903F0938A03662708
:101C4E0077270E94B621A6EFB8E284E991E40E94BC
:101C5E004022A9E8B3E00E947D21ED93FC93E09130
:101C6E006205F0916305A0918903B0918A03EA0F92
:101C7E00FB1FE0938903F0938A03A0918903B0912F
:101C8E008A03A030E4E0BE0710F40C94540EEFEF7C
:101C9E00F3E0E0938903F0938A03E091AD05EF70D2
:101CAE00E0931B03ADEAB5E0EC91E295EF70EC9397
:101CBE00AA2011F00C94760EE091AD05EF70E09332
:101CCE007303A5E0EA02F001E0937303A09173039E
:101CDE00A13010F00C94760EE1E0E0937303E1E096
:101CEE00EA1511F00C94800EE091AD05EF70E093C3
:101CFE005805A091AE05A13010F40C948C0EE09115
:101D0E00AE05F0E0E883F98304C0EDE1F0E0E8838E
:101D1E00F983A091AF05B0E0E7E00E941123E13016
:101D2E00A0E0FA0711F00C94A00EE091AF05EF774A
:101D3E00EC8BA091B005B0E0E7E00E941123E130FA
:101D4E00A0E0FA0711F00C94B00EE091B005EF7719
:101D5E00EB8BEC8DE03011F00C94B90EE091690331
:101D6E00E0936803689422F8EFE34E2EE1E0EE2E46
:101D7E00A0917403E0E00E9429230E2EE7E00E945A
:101D8E002923E02911F40C94CF0EE1E0E0937403C3
:101D9E00E1E06E2EE0E0EF8BAF89A03110F00C94F5
:101DAE00E20EEF89F0E0EE55FA4FA0E0A083EF8946
:101DBE00EF5FEF8BF1CFE0E0E093CA05E0936703AE
:101DCE00A091CA05E0E10E9433230E2EA091A20538
:101DDE00EBE60E9429230E22A091CA05E0E10E94A3
:101DEE003D23E02911F40C94120FE0E0EF8BAF8944
:101DFE00A03110F00C940D0FEF89F0E0EE55FA4F74
:101E0E00A0E0A083EF89EF5FEF8BF1CFE0E0E093EE
:101E1E00CA05E0936703AE89A13011F00C94180F38
:101E2E00F69AA0918405B0918505EAE0F0E00E9453
:101E3E005A230E2EE6EFFFEF0E9460230E22AE898C
:101E4E00E0E00E9429230E22A0916805B091690559
:101E5E00E1E0F0E00E945A23E02111F40C94380FD7
:101E6E00F698A0918405B0918505EAE0F0E00E9415
:101E7E0060230E2EE6EFFFEF0E945A23E02911F4A5
:101E8E000C944A0FF69AF6990BC0E0E0E0936803C3
:101E9E00E0936805E0936905E0936A05E0936B05AE
:101EAE00E0917E05F0917F05A4E9B5E00E941F2325
:101EBE000E94B6210E941724A0914205B0914305BD
:101ECE00A036EAEEBE0710F00C94760FE0914205B4
:101EDE00F09143053196E0934205F0934305A091AE
:101EEE004605B0914705A031E7E2BE0710F40C9409
:101EFE008C0FE0E0E0938405E0938505E0E1F7E2E6
:101F0E00E0934805F093490535C023FE19C0E091D2
:101F1E004805F091490566277727A1E5B5E282E0ED
:101F2E0090E00E94F123E0938405F0938505A0E9EB
:101F3E00B5E00E941F230E94B6210E9417241AC0EA
:101F4E00E0914805F091490566277727AFEABAED8B
:101F5E008DEF9FEF0E94F123E0938405F0938505AA
:101F6E000E94FD22A0E9B5E00E941F230E94B62127
:101F7E000E941724E0914805F091490566277727BE
:101F8E00A0E0B0EC8EE190E00E94F123ACE9B5E068
:101F9E000E94B6210E941724E0919C05F0919D05A8
:101FAE0060919E0570919F05A4E5B5E00E947D218C
:101FBE00ED93FC93A0915405B0915505A130E0EE40
:101FCE00BE0710F40C94F10FE0E0F0EEE093540530
:101FDE00F0935505E881F981A0919005B091910596
:101FEE008091920590919305662777270E94B621DE
:101FFE000E948E22E0939005F093910560939205D6
:10200E0070939305E0919405F09195056091960576
:10201E0070919705A0E0B0E68FE195E40E948E22C4
:10202E00A0919005B09191058091920590919305A4
:10203E000E944022E0939005F093910560939205E3
:10204E0070939305A0919005B091910580919205A2
:10205E0090919305E0E0F0E06EE773E40E94D322E6
:10206E0009F010F40C944310E0939005F093910551
:10207E006093920570939305E0919005F091910510
:10208E006091920570919305A1EAB5E00E947D21C1
:10209E00EC93EFE3E41511F00C9471104424E0E09E
:1020AE00E0938303E0938403A0916805B0916905E2
:1020BE00E0E0F0E00E9442230E2EA0918205B09146
:1020CE008305E0E0F0E00E944223E02111F40C943D
:1020DE007110F398A0916805B0916905E0E0F0E009
:1020EE000E9460230E2EA0918205B0918305E0E040
:1020FE00F0E00E9442230E22A0E0F699A1E0E1E07A
:10210E000E942923E02111F40C94A110E091830385
:10211E00F09184033196E0938303F0938403A091AE
:10212E008303B0918403A83EE3E0BE0711F00C9444
:10213E00A110F09AE0910903E03011F00C94C71150
:10214E00A0916803E1E00E9429230E2EE2E00E9496
:10215E002923E02911F40C94C810A0916C05B091BC
:10216E006D05E0916A05F0916B05EA1BFB0BDF0133
:10217E00E2E0F0E00E94C723E0938605F093870526
:10218E0021C0A0915E05B0915F05E4E0F0E00E94F1
:10219E00C723E0938605F0938705A0915F05AA23D8
:1021AE0012F00C94E910E0915E05F0915F050E942B
:1021BE00FD22DF01E4E0F0E00E94C723E0938605F4
:1021CE00F0938705A0916405B0916505ECEEFFEFE5
:1021DE000E9460230E2EE0E0F0E00E944E23E021EC
:1021EE0011F40C940911E0916405F09165050E94BB
:1021FE00FD22DF01E2E0F0E00E94C723E0938605B6
:10220E00F0938705A0916405B0916505E4E1F0E0D7
:10221E000E945A230E2EE0E0F0E00E946023E0219F
:10222E0011F40C942211E2E0F0E00E94C723E09337
:10223E008605F0938705A0917E05B0917F05E0910C
:10224E004A05F0914B053A960E9466230E2EA091F8
:10225E007E05B0917F05E0914A05F0914B050E94F5
:10226E006C23E02111F40C944A11E0917E05F0915B
:10227E007F05A0914A05B0914B05EA1BFB0BE0933D
:10228E008605F0938705A0917E05B0917F051A967D
:10229E00E0914A05F0914B050E946C230E2EA09101
:1022AE007E05B0917F05E0914A05F0914B050E94A5
:1022BE006623E02111F40C947211E0917E05F091E9
:1022CE007F05A0914A05B0914B05AE1BBF0BA093A5
:1022DE008605B0938705E0917A03A0916805B091C9
:1022EE006905F0E00E945A231E2EA0916803E0E0DB
:1022FE000E9429230E2EE3E00E942923E029E121EA
:10230E0011F40C949B11A0917A03BB27E091680500
:10231E00F0916905AE1BBF0BE2E0F0E00E94C7230F
:10232E00E0938605F0938705E0916C05F0916D05BD
:10233E00A0916A05B0916B050E945A231E2EA091A2
:10234E006803E1E00E9429230E2EE2E00E94292379
:10235E00E029E12111F40C94C711A0916A05B09106
:10236E006B05E0916C05F0916D05EA1BFB0BDF012F
:10237E00E4E0F0E00E94C723E0938605F093870522
:10238E00A0910903A13011F00C942312EAE0F0E0C1
:10239E00E0938605F0938705A0917E05B0917F05A9
:1023AE00E0914C05F0914D053A960E9466230E2E53
:1023BE00A0917E05B0917F05E0914C05F0914D0501
:1023CE000E946C23E02111F40C94FB11E0917E0528
:1023DE00F0917F05A0914C05B0914D05EA1BFB0BCA
:1023EE00E0938605F0938705A0917E05B0917F0559
:1023FE001A96E0914C05F0914D050E946C230E2E1D
:10240E00A0917E05B0917F05E0914C05F0914D05B0
:10241E000E946623E02111F40C942312E0917E05B4
:10242E00F0917F05A0914C05B0914D05AE1BBF0BF1
:10243E00A0938605B0938705A0918705AA2312F075
:10244E000C943312E0918605F09187050E94FD22CF
:10245E00E0938605F0938705A0918605B0918705D8
:10246E001B9714F40C944112EAE0F0E0E093860519
:10247E00F0938705E0918605F0918705309711F06E
:10248E000C944F12E1E0F0E0E0938605F09387059F
:10249E00E0918605A0918203EA0FE0938203A0915A
:1024AE006805B0916905E0E0F0E00E9460230E2E11
:1024BE00A0E0F699A1E0E1E00E942923E02111F4C9
:1024CE000C949114A0916803E0E00E9429230E2E33
:1024DE00E3E00E9429230E2AE0917A03A091680579
:1024EE00B0916905F0E00E945423E0211E2EA091C8
:1024FE006C05B0916D05E1E0F0E00E945A230E2EBE
:10250E00A0916805B0916905E0E0F0E00E946023BB
:10251E00E0211E2AA0916803E1E00E9429230E2EDD
:10252E00E0916C05F0916D05A0916A05B0916B0577
:10253E000E946023E0211E2AA0916803E2E00E941F
:10254E0029230E2EE0917A03A0916805B0916905BA
:10255E00F0E00E9460230E22E0916C05F0916D0573
:10256E00A0916A05B0916B050E946023E021E129DC
:10257E0011F40C94D513A0915E05B0915F05E0E0C7
:10258E00F0E00E945A230E2EA0916405B0916505CD
:10259E00E0E0F0E00E945A230E22A0917E05B09159
:1025AE007F05E0914A05F0914B050E946C23E021D6
:1025BE0011F40C948513A0917A03AE3F10F00C9495
:1025CE006613E5E0EC1510F00C946513A0918203F0
:1025DE00AA3010F40C946513E0917A03EF5FE09348
:1025EE007A03A0917E05B0917F05E0914A05F091A6
:1025FE004B053A960E946C230E2EE0917A03F0E082
:10260E00A0916805B0916905AE1BBF0BE4E1F0E047
:10261E000E9460230E22A0915E05B0915F05ECEE44
:10262E00FFEF0E945A230E22A0916405B09165051A
:10263E00EEECFFEF0E945A230E22A0916803E1E018
:10264E000E942E23E0211E2EA0917E05B0917F05C3
:10265E00E0914A05F0914B053A960E946C230E2E9E
:10266E00A0916C05B0916D05E0916A05F0916B0536
:10267E00EA1BFB0BDF01E2E3F0E00E9460230E2277
:10268E00A0916405B0916505EEECFFEF0E945A2310
:10269E000E22A0916803E1E00E942923E021E129A6
:1026AE0011F40C946513A0917A03AC3F10F00C94C6
:1026BE006513E0917A03EE5FE0937A031EC0E0911A
:1026CE001B03A0911C030E9438230E2EA0916803B9
:1026DE00E0E00E943D230E22E3E00E9438230E220A
:1026EE00AB2DE2E30E942923E02111F40C94841314
:1026FE00E0911C03EF5FE0931C0350C0A0917E0598
:10270E00B0917F05E0914A05F0914B05EA17FB0762
:10271E0010F40C94C113A0916C05B0916D05E1E01D
:10272E00F0E00E945A230E2EA0917A03EEEF0E9443
:10273E003823E02111F40C94A913E0917A03EF5F92
:10274E00E0937A03A0916C05B0916D05E1E0F0E0A5
:10275E000E9460230E2EA0917A03E0E00E943D239A
:10276E00E02111F40C94C013E0917A03E150E09350
:10277E007A0314C0A0918203E9E00E943D230E2E3D
:10278E00A0917A03E0E00E943D23E02111F40C9425
:10279E00D513E0917A03E150E0937A03A091680398
:1027AE00E1E00E9429230E2EE2E00E9429230E2A48
:1027BE00E0916C05F0916D05A0916A05B0916B05E5
:1027CE000E945A23E02111F40C944214A0917A0332
:1027DE00E1E00E943D230E2EA0911C03E0E00E943A
:1027EE002923E02111F40C942614A0918203AA301F
:1027FE0010F40C942514E0917A03E150E0937A03DF
:10280E00A0917A03E2E00E943D230E2EA0916A056C
:10281E00B0916B05E0916C05F0916D05EA1BFB0B19
:10282E00DF01E2E3F0E00E946023E02111F40C945A
:10283E002514E0917A03E250E0937A031CC0A09134
:10284E001C03E0E00E943D230E2EAB2DE2E30E941E
:10285E0029230E22A0916C05B0916D05EBEFFFEFD1
:10286E000E946023E02111F40C944214E0911C03A9
:10287E00E150E0931C03A0916803E1E00E942E2337
:10288E000E2EE0917A03A0916805B0916905F0E0F3
:10289E000E945A230E22A0918203E9E00E943D235A
:1028AE00E02111F40C949014E1E0E91511F00C9470
:1028BE007914A0916C05B0916D05129714F40C94D7
:1028CE007814E0917A03E150E0937A03A0916C05BD
:1028DE00B0916D05559714F40C947814E250E09372
:1028EE007A0317C0E0917A03E150E0937A03A09146
:1028FE007A03BB27E0916805F0916905AE1BBF0B0B
:10290E00559714F40C949014E0917A03E250E093EE
:10291E007A031CC0A0916C05B0916D05E1E0F0E06A
:10292E000E945A230E2EA0911C03E0E00E943D232C
:10293E000E22AB2DE2E30E942923E02111F40C9428
:10294E00AD14E0911C03E150E0931C03A0916C05C3
:10295E00B0916D05E2E0F0E00E945A230E2EEEEFEC
:10296E00FFEF0E9460230E2AA0918405B091850589
:10297E00E0E0F0E00E9442230E22A0917805B09193
:10298E007905E4E6F0E00E9460230E22A0E0F499BF
:10299E00A1E0E0E00E9429230E22A0E0F099A1E040
:1029AE00E0E00E9429230E22A0E0F399A1E0E0E0EE
:1029BE000E942923E02111F40C94F814A0917203C3
:1029CE00AA3F10F00C94F114E0917203EF5FE093C4
:1029DE00720307C027FE04C0E1E0E093090301C0C3
:1029EE00F39AA0910903E1E00E9429231E2EA091E3
:1029FE007805B0917905E4E6F0E00E945A230E2E98
:102A0E00A0E0F499A1E0E1E00E9429230E2AA0E0C3
:102A1E00F099A1E0E1E00E9429230E2AA0E0F399AB
:102A2E00A1E0E1E00E9429230E2AA0E027FCA1E00C
:102A3E00E0E00E9429230E2AA0918405B09185051D
:102A4E00E0E0F0E00E944823E029E12111F40C942B
:102A5E003715E0E0E0937203E0930903E0937A0305
:102A6E00A0910903E1E00E9429230E2EA09182037A
:102A7E00E9E00E943D23E02111F40C94A015A091F1
:102A8E007A03E0EF0E9438231E2EE0918C05F09120
:102A9E008D0560918E0570918F050E940123A09186
:102AAE006C05B0916D050E9424230E947A230E2E90
:102ABE00A0917E05B0917F05E0914C05F0914D05FA
:102ACE000E946623E021E12111F40C947315E0912C
:102ADE007A03EF5FE0937A03A0917A03E0E00E941D
:102AEE003D231E2EE0918C05F0918D0560918E0593
:102AFE0070918F050E940123A0916C05B0916D0518
:102B0E000E9424230E9472230E2EA0917E05B09166
:102B1E007F05E0914C05F0914D050E946C23E02954
:102B2E00E12111F40C94A015E0917A03E150E093A9
:102B3E007A03A0918203AA3010F40C94AB15E091A5
:102B4E008203EA50E0938203A0911C03A13010F49B
:102B5E000C94B515E1E0E093080303C0E0E0E093C8
:102B6E000803E0911B03A0911C03EA1711F00C94CB
:102B7E00C315E1E0DE2E01C0DD24A0916803E0E084
:102B8E000E9429230E2EE3E00E942923E02911F44E
:102B9E000C94D415E0E0E0931C03A0917A03BB27BC
:102BAE00E091A105F0E0AE1BBF0BE0915805F0E0FF
:102BBE00E7FDFFEF0E94AA23DF01E0E4F0E00E94B0
:102BCE00C723E0935705A0915705A03014F00C943D
:102BDE00F315E0E0E0935705A0915705B0E0A7FD8F
:102BEE00BFEFE0911C03F0E0EA0FFB1F0E941F23D2
:102BFE000E94B621A6E6B6E686E490E40E94F02195
:102C0E00A0919805B091990580919A0590919B0598
:102C1E000E94E921ADECBCEC8CE49DE30E944022C5
:102C2E00A0919805B091990580919A0590919B0578
:102C3E000E94F021E0939805F093990560939A0510
:102C4E0070939B05A0919805B091990580919A0576
:102C5E0090919B05E0E0F0E060E771E40E94D322E2
:102C6E0009F010F40C944316E0939805F09399052F
:102C7E0060939A0570939B05A0919B05AA2312F071
:102C8E000C945216E0E0E0939805E0939905E093DA
:102C9E009A05E0939B05E0919805F0919905609156
:102CAE009A0570919B05A9E5B5E00E947F21EC93F2
:102CBE00E1E3EB1510F00C946516BB24B394E09190
:102CCE006B03F0E0E0938703F0938803E0916B03CE
:102CDE00F0E0B996A0918703B0918803AE17BF07B5
:102CEE0010F00C94AD16A335E0E0BE0710F00C9476
:102CFE00A516E0918703F0918803E151FB4FA08167
:102D0E00B0E0E0917A03F0E00E94AA230E941A2319
:102D1E00E0934405F0934505A0918703B091880395
:102D2E00E4EAF0E0EA1BFB0BE251FC4F0F01A2516B
:102D3E00BC4FE0914405EC93D001EC93A7E8B3E0CF
:102D4E00ED91FD913196FE93EE93C0CFE0916B0322
:102D5E00E75DE0936B03A0916B03A33510F40C9425
:102D6E00BB16E0E0E0936B03A0918503B091860360
:102D7E00E6E9F0E00E9442230E2EA0914205B091AA
:102D8E004305E4EFF1E00E946C23E02111F40C9472
:102D9E00D216689420F820FE53C0E0E0E093680558
:102DAE00E0936905E0936A05E0936B057394A72D94
:102DBE00EAE00E943D230E2EA0918D03B0918E036A
:102DCE00EFEFF0E00E946623E02111F40C94271738
:102DDE007724E0918D03F0918E033196E0938D036D
:102DEE00F0938E03A0918D03B0918E03EFEFF0E080
:102DFE00EA1BFB0B0F01EFEFF0E0EA1BFB0BD00120
:102E0E000E948223DF01EFEFF0E00E94B4230F0156
:102E1E00A0918D03B0918E03EFEFF0E0EA1BFB0B58
:102E2E00D0010E948223DF01EFEFF0E00E94B42375
:102E3E00AFEFB0E0AE1BBF0BA0938205B09383053E
:102E4E00A0918405B0918505E2E0F0E00E945A233E
:102E5E000E2EEEEFFFEF0E9460230E22A0E020FC6C
:102E6E00A1E0E1E00E942923E02111F40C94461721
:102E7E00E89420F8E0E0E0938D03E0938E03A091B8
:102E8E006805B0916905E0E0F0E00E9442230E2E45
:102E9E00A0918205B0918305E0E0F0E00E9442230C
:102EAE00E02111F40C946B17F098E0E0E0938303AB
:102EBE00E0938403F49B03C0E1E0E0936F03F39B84
:102ECE0003C0E1E0E0937003A0916805B09169053D
:102EDE00E0E0F0E00E9442230E2EA0918205B09118
:102EEE008305E0E0F0E00E9442230E22A0916C05E3
:102EFE00B0916D05E5E0F0E00E945A230E22EBEF53
:102F0E00FFEF0E946023E02111F40C94C917A091E9
:102F1E008B03B0918C03A83BEBE0BE0710F00C9432
:102F2E00A217E0918B03F0918C033196E0938B0303
:102F3E00F0938C0326C0A0916C05B0916D050E9494
:102F4E00462414F00C94B417E0915C05F0915D05E5
:102F5E003196E0935C05F0935D05A0916D05AA2373
:102F6E0012F00C94C317E0915C05F0915D0531975A
:102F7E00E0935C05F0935D05E0E0E0938B03E09356
:102F8E008C0305C0E0E0E0938B03E0938C03A0E09C
:102F9E00F199A1E0E1E00E9429230E2EA0E0F29922
:102FAE00A1E0E1E00E942923E02911F40C94E0173E
:102FBE00F49AE0917A03F0E00E941F230E94B6215A
:102FCE00ADECBCEC8CEC9DE30E944022A0E8B3E09B
:102FDE000E947D21EC93A0E0F499A1E0E0E00E9434
:102FEE0029230E2EA0E0F099A1E0E0E00E94292313
:102FFE000E22A0E0F399A1E0E0E00E942923E02157
:10300E0011F40C94751CA0918205B0918305E0E03B
:10301E00F0E00E9442230E2EA0916805B091690542
:10302E00E0E0F0E00E9460230E22A0917803E3E03E
:10303E000E9438230E22A0E025FCA1E0E1E00E94D0
:10304E002923E0211E2EA0918205B0918305E0E098
:10305E00F0E00E9442230E2EA0916805B091690502
:10306E00E0E0F0E00E9442230E22EA2DA92D0E94FC
:10307E002E23E021E12911F40C94EC1AE5E0EC1575
:10308E0010F00C94EB1A9A2CE0911A03E03011F028
:10309E000C949919E3E0E0930B03E6E0E0930C0344
:1030AE00E2E0E0930D03E5E0E0930E03E1E0E09350
:1030BE000F03E4E0E0931003E1E0E093780399203E
:1030CE0011F00C940D19A0917A03A13010F40C9408
:1030DE008418E0917303F0E0A0916C05B0916D053A
:1030EE000E94AA23DF01E0917A03F0E00E94C72339
:1030FE00E0935005F093510505C0E0E0E0935005D4
:10310E00E0935105A0915005B0915105A030E1E03A
:10311E00BE0710F40C949718EFEFE093610304C010
:10312E00E0915005E0936103E0917A03E093CB03C5
:10313E00E093C903E093AF03E093AE03E0939803EB
:10314E00E0939403EFEFE093D303E093D103E09386
:10315E00B703E093B603E093A003E0939C03E0E093
:10316E00E093D003E093CE03E093B903E093B8036A
:10317E00E093A103E0939D03E0939603E093950300
:10318E00E0939903E0939703E093B203E093B003C7
:10319E00E093B103E093AD03E093C803E093C7035C
:1031AE00E093CA03E093C603A0916C05B0916D0540
:1031BE00A436E0E0BE0714F00C94F418E4E2E093B9
:1031CE00E103E093DF03E9E0E093E403E093E0033F
:1031DE00E2E1E093E303E093E203A0916C05B0918A
:1031EE006D05A739E0E0BE0714F40C940D19EFE25B
:1031FE00E093E403E093DF03EFE1E093E303E09376
:10320E00E003E7E3E093E203E093E103E4E2E0931B
:10321E00E903E093E703E9E0E093EC03E093E803CE
:10322E00E2E1E093EB03E093EA03A92DE1E00E94D3
:10323E0029230E2EA0E022FCA1E0E1E00E9429232A
:10324E00E02111F40C949919E0E0E0936103E89405
:10325E0022F8EFE3E093E403E093E303E093E20369
:10326E00E093E103E093E003E093DF03E0E0E0931B
:10327E005703E0934F03E0934703E0935C03E0931F
:10328E005503E0934A03E9E2E0935B03E0935103B5
:10329E00E0934803E2E5E0935D03E0935203E0938D
:1032AE004C03EBE7E0935903E0935003E0934B0399
:1032BE00E4EAE0935A03E0935403E0934D03EDECFC
:1032CE00E0935803E0935303E0934903E0E0E09367
:1032DE005E03E0935603E0934E03A0918405B091F4
:1032EE0085051A9714F00C949919E0917403F0E087
:1032FE00E95BFC4FE081A0915905EA0FE093900342
:10330E00E0917403F0E0E15BFC4FE081EA0FE093A3
:10331E009103E0917403F0E0E95AFC4FE081EA0F6B
:10332E00E0939203A0911A03A13011F00C94EA1AC3
:10333E00E5E0E0930B03E3E0E0930C03E1E0E093C0
:10334E000D03E6E0E0930E03E4E0E0930F03E2E00A
:10335E00E0931003E0937803992011F00C946A1A0D
:10336E00A0917A03A13010F40C94D119E09173035B
:10337E00F0E0A0916C05B0916D050E94AA23DF01CB
:10338E00E0917A03F0E00E94C723E0935005F0939A
:10339E00510505C0E0E0E0935005E0935105A09182
:1033AE005005B0915105A030E1E0BE0710F40C9429
:1033BE00E419EFEFE093610304C0E0915005E09350
:1033CE006103E0917A03E093C803E093C603E093B0
:1033DE00B103E093B003E0939903E0939503E0E02B
:1033EE00E093D303E093D103E093B703E093B603E6
:1033FE00E093A003E0939C03EFEFE093D003E09300
:10340E00CE03E093B903E093B803E093A103E093F6
:10341E009D03E0E0E0939803E0939703E093960317
:10342E00E0939403E093B203E093AF03E093AE0313
:10343E00E093AD03E093CB03E093CA03E093C9039B
:10344E00E093C703A0916C05B0916D05A436E0E042
:10345E00BE0714F00C94421AE9E0E093E303E09304
:10346E00DF03E2E1E093E103E093E003E4E2E093C3
:10347E00E403E093E203A0916C05B0916D05A739CA
:10348E00E0E0BE0714F40C945B1AEFE2E093E40361
:10349E00E093DF03EFE1E093E303E093E003E7E380
:1034AE00E093E203E093E103E9E0E093EB03E093C2
:1034BE00E703E2E1E093E903E093E803E4E2E0935B
:1034CE00EC03E093EA03A92DE1E00E9429230E2EDE
:1034DE00A0E022FCA1E0E1E00E942923E02111F40A
:1034EE000C94EA1AE0E0E0936103E89422F8EFE32B
:1034FE00E093E403E093E303E093E203E093E1035C
:10350E00E093E003E093DF03E0E0E0935703E09302
:10351E004F03E0934703E0935C03E0935503E0937E
:10352E004A03E9E2E0935803E0935303E09349031F
:10353E00E2E5E0935A03E0935403E0934D03EBE787
:10354E00E0935903E0935003E0934B03E4EAE093D6
:10355E005D03E0935203E0934C03EDECE0935B03C9
:10356E00E0935103E0934803E0E0E0935E03E093C1
:10357E005603E0934E03A0918405B0918505E6EFC6
:10358E00FFEFEA17FB0714F00C94EA1AE0917403AC
:10359E00F0E0E95BFC4FE081A0915905EA0FE09362
:1035AE009003E0917403F0E0E15BFC4FE081EA0FE1
:1035BE00E0939103E0917403F0E0E95AFC4FE0814F
:1035CE00EA0FE093920301C0C394A0918205B091DB
:1035DE008305E0E0F0E00E9442230E2EA0916805E4
:1035EE00B0916905E0E0F0E00E9442230E22A09126
:1035FE000903E0E00E942923E0211E2EA09178030A
:10360E00E3E00E9429230E2EA0916805B091690572
:10361E00E0E0F0E00E946023E0211E2AA0918205E6
:10362E00B0918305E0E0F0E00E9442230E2EA0E070
:10363E0025FCA1E0E0E00E9429230E22A0910903BF
:10364E00E0E00E942923E021E12911F40C94AF1B44
:10365E00CC24E091A105E0937A03A0911A03E0E057
:10366E000E9429230E2EA0918405B0918505E0E0DD
:10367E00F0E00E946023E0211E2EA0911A03E1E0EB
:10368E000E9429230E2EA0918405B0918505E0E0BD
:10369E00F0E00E945A23E021E12911F40C945C1B06
:1036AE00E091A105E0937A0303C0E0E0E0937A0392
:1036BE00E0E0E09378039A2C689422F8E0939B0361
:1036CE00E0939A03E0939903E0939803E0939703B2
:1036DE00E0939603E0939503E0939403E0939303B2
:1036EE00E093B403E093B303E093B203E093B1032A
:1036FE00E093B003E093AF03E093AE03E093AD032A
:10370E00E093AC03E093CD03E093CC03E093CB03C3
:10371E00E093CA03E093C903E093C803E093C703A1
:10372E00E093C603E093C503E093DE03E093DF036B
:10373E00E093E003E093E103E093E203E093E3031D
:10374E00E093E403E093E503E093E603E093610383
:10375E00A0918205B09183050E94462414F00C942A
:10376E00741CCC24A0917803A33010F00C94C21BCF
:10377E00E0E0E0937A03E3E0E0930B03E6E0E0930E
:10378E000C03E2E0E0930D03E5E0E0930E03E1E0CD
:10379E00E0930F03E4E0E0931003689422F8992479
:1037AE00E3E0E0937803E0E0E0936103A091090386
:1037BE00A13011F00C941B1CE0939B03E0939A0331
:1037CE00E0939903E0939503E0939803E0939703B6
:1037DE00E0939603E0939403E0939303EFEFE0936B
:1037EE00CD03E093CC03E093CB03E093CA03E093C5
:1037FE00C903E093C803E093C703E093C603E093C5
:10380E00C503E093B403E093B303E093B203E093F4
:10381E00B103E093B003E093AF03E093AE03E09304
:10382E00AD03E093AC0338C0E0918205E093CD0385
:10383E00E093CC03E093CB03E093CA03E093C90378
:10384E00E093C803E093C703E093C603E093C50378
:10385E00E093B403E093B303E093B203E093B103B8
:10386E00E093B003E093AF03E093AE03E093AD03B8
:10387E00E093AC03E0939B03E0939A03E0939903E8
:10388E00E0939503E0939803E0939703E0939603F8
:10389E00E0939403E0939303E7E0E093E603E09371
:1038AE00E503E093E403E093E303E093E203E093A4
:1038BE00E103E093E003E093DF03E093DE03A091E6
:1038CE007E05B0917F05E0914C05F0914D05EA170C
:1038DE00FB0710F40C94741CF59A99C0E0E0E09389
:1038EE006103E0931C03E0937A03E0939B03E09360
:1038FE009A03E0939903E0939803E0939703E09380
:10390E009603E0939503E0939403E0939303E0937F
:10391E00B403E093B303E093B203E093B103E093F7
:10392E00B003E093AF03E093AE03E093AD03E093F7
:10393E00AC03E093CD03E093CC03E093CB03E09391
:10394E00CA03E093C903E093C803E093C703E0936F
:10395E00C603E093C503E093DE03E093DF03E09339
:10396E00E003E093E103E093E203E093E303E093EB
:10397E00E403E093E503E093E603A0916805B091BC
:10398E006905E0E0F0E00E9460230E2EA091820512
:10399E00B0918305E0E0F0E00E946023E02911F48D
:1039AE000C940E1DA0916F03E1E00E9429230E2EB0
:1039BE00A0917003E1E00E942923E02911F40C94F8
:1039CE000E1DE091A105E0937A03F498E0E0E093F8
:1039DE006F03F398E0937003E1EAE4BDE1E8E0934E
:1039EE00B000E1E0E91511F00C940E1DEFE3E09349
:1039FE00E503E093E403E093E303E093E203E09353
:103A0E00E103E093E003E093DF03E093DE03E09154
:103A1E008205F0918305309711F00C94171DF598DF
:103A2E00003011F00C941D1D54985C98013011F06B
:103A3E000C942C1D549AE0917E03EE1FE0E0EE1FD5
:103A4E00E17011F45C9801C05C9A023011F00C9494
:103A5E00391D549AE0917E03E295E17011F45C9861
:103A6E0001C05C9A033011F00C943F1D549A5C9A7D
:103A7E00303011F00C94501DE0E0E51510F00C9470
:103A8E004C1D229A50928A0004C02298E0E0E093E6
:103A9E008A00313011F00C94601D229AE0917E0361
:103AAE00EE1FE0E0EE1FE170A52DEA02F001E093BB
:103ABE008A00323011F00C946E1D229AE0917E0332
:103ACE00E295E170A52DEA02F001E0938A00333011
:103ADE0011F00C94931D229AE0917E03E295EF7003
:103AEE00AE2FE0917E03E295EF70E695EA23AE2FBE
:103AFE00E0917E03E295EF70E695E695EA23AE2F10
:103B0E00E0917E03EE1FE0E0EE1FEA23E170A52DAB
:103B1E00EA02F001E0938A00203011F00C94A41D0B
:103B2E00E0E0E81510F00C94A01D219A8092880018
:103B3E0004C02198E0E0E0938800213011F00C944D
:103B4E00B41D219AE0917E03EE1FE0E0EE1FE170BE
:103B5E00A82DEA02F001E0938800223011F00C94B7
:103B6E00C21D219AE0917E03E295E170A82DEA0232
:103B7E00F001E0938800233011F00C94E71D219A98
:103B8E00E0917E03E295EF70AE2FE0917E03E29519
:103B9E00EF70E695EA23AE2FE0917E03E295EF708B
:103BAE00E695E695EA23AE2FE0917E03EE1FE0E068
:103BBE00EE1FEA23E170A82DEA02F001E0938800DF
:103BCE00A0E0B0E00E942924A12F0E9429230E2EEE
:103BDE00A0916C03E1E00E942923E02111F40C94E2
:103BEE003121E0E0E0936C03E0917E05F0917F05DA
:103BFE00E0936605F0936705E0917805F0917905FD
:103C0E00E0937005F0937105E0916C05F0916D05F0
:103C1E000E941F230E94B621A7E1B9ED8EE09FE31B
:103C2E000E944022AAE5B5E00E947F21ED93FC930D
:103C3E00E0917A03E0937C03A0917C03E0E00E9484
:103C4E003D230E2EA0910903E0E00E942923E021DE
:103C5E0011F40C947A1EA0916D05AA2312F40C9403
:103C6E00581EE0915A05F0915B050E941F230E9499
:103C7E00B621A0E0B0E08CEC91E40E944022DF017E
:103C8E00CB01E0917C03F0E00E941F230E94B6213D
:103C9E000E948E22AEE6B5E00E947F21ED93FC934A
:103CAE0021C0E0915A05F0915B050E94FD220E9411
:103CBE001F230E94B621A0E0B0E08CEC91E40E949C
:103CCE004022DF01CB01E0917C03F0E00E941F2334
:103CDE000E94B6210E948E22AEE6B5E00E947F21A0
:103CEE00ED93FC9305C0E0E0E0936E05E0936F0565
:103CFE00A0910903A13011F00C94BE1EA0916D0588
:103D0E00AA2312F00C94BE1EE0915A05F0915B05A9
:103D1E000E94FD220E941F230E94B621A0E0B0E067
:103D2E008CEC91E40E9440227F936F93FF93EF936C
:103D3E00E0917A03F0E0AFEFB0E00E942224EA1B9C
:103D4E00FB0BAF91BF918F919F910E941F230E94F9
:103D5E00B6210E948E22A0E0B0E080E09FE30E9498
:103D6E00F021AEE6B5E00E947F21ED93FC93EFE0EB
:103D7E00EB83E0E0EC83ED83E98DE03011F00C9401
:103D8E00CB1EE091A005EC83A98DA13011F00C940F
:103D9E00D31EE0917A03EC83A98DA23011F00C941E
:103DAE00DB1EE091A105EC83A98DA33011F00C94DC
:103DBE00ED1EE0919805F091990560919A0570912C
:103DCE009B05DE0114960E947D21EC93A98DA430F3
:103DDE0011F00C94F51EE0911C03EC83A98DA53017
:103DEE0011F00C94FD1EE0915905EC83A98DA630BF
:103DFE0011F00C940C1FE0916605F09167050E947E
:103E0E001A23EC83E0916605ED83A98DA83011F09D
:103E1E000C94391FFE0134960F01A081E0E04A99FF
:103E2E00E1E0EA0FD001EC93DE011496EC91EE0F77
:103E3E00EC93FE0134960F01A081E0E01D99E1E0C4
:103E4E00EA0FD001EC93DE011496EC91EE0FEC9399
:103E5E00FE0134960F01A081E0E01C99E1E0EA0F2B
:103E6E00D001EC93A98DA93011F00C948C1FFE019A
:103E7E003496E082DE011496EC91EE0FEC93FE0187
:103E8E0034960F01A081E0E04B99E1E0EA0FD001FA
:103E9E00EC93DE011496EC91EE0FEC93FE0134964A
:103EAE000F01A081E0E0F099E1E0EA0FD001EC9380
:103EBE00DE011496EC91EE0FEC93FE0134960F0199
:103ECE00A081E0E01999E1E0EA0FD001EC93DE0168
:103EDE001496EC91EE0FEC93FE0134960F01A08137
:103EEE00E0E01A99E1E0EA0FD001EC93DE011496BE
:103EFE00EC91EE0FEC93FE0134960F01A081E0E001
:103F0E004C99E1E0EA0FD001EC93A98DAA3011F0A3
:103F1E000C949B1FE0917005F09171050E941A237D
:103F2E00EC83E0917005ED83E0910903EE83DE01F1
:103F3E001696EC91EE0FEE0FEC93FE0136960F01F6
:103F4E00A081E0916E05F0916F050E941A23E37037
:103F5E00EA0FD001EC93DE011696EC91EE0FEE0F08
:103F6E00EC93FE0136960F01A081E0915A05F09177
:103F7E005B050E941A23E370EA0FD001EC93DE0179
:103F8E001696EC91EE0FEE0FEC93FE013696BF01F6
:103F9E000080A0E0B0E00E942924E00DDB01EC934C
:103FAE00E0915A05EF83E0916E05E887E0917A0380
:103FBE00E987E0918405F09185050E941A23EA872E
:103FCE00E0918405EB87FE013C96E082DE011C96B3
:103FDE00EC91EE0FEC93FE013C960F01E081A09167
:103FEE006403EA0FD001EC93DE011C96EC91EE0F08
:103FFE00EC93FE013C960F01A081E0E0F599E1E023
:10400E00EA0FD001EC93DE011C96EC91EE0FEC93CF
:10401E00FE013C960F01A081E0E0F399E1E0EA0F8A
:10402E00D001EC93DE011C96EC91EE0FEC93FE01A9
:10403E003C960F01A081E0E0F499E1E0EA0FD00197
:10404E00EC93DE011C96EC91EE0FEC93FE013C9688
:10405E000F01A081E0E01999E1E0EA0FD001EC93A5
:10406E00DE011C96EC91EE0FEC93FE013C960F01D7
:10407E00A081E0E01A99E1E0EA0FD001EC93DE01B5
:10408E001C96EC91EE0FEC93FE013C960F01A08175
:10409E00E0E04C99E1E0EA0FD001EC93FE013D9691
:1040AE00D082DE011D96EC91EE0FEC93FE013D9653
:1040BE000F01E081A0910803EA0FD001EC93DE011D
:1040CE001D96EC91EE0FEE0FEC93FE013D960F0157
:1040DE00A081E0917605F09177050E941A23EA0FF0
:1040EE00D001EC93DE011D96EC91EE0FEE0FEC93EA
:1040FE00FE013D960F01A081E0917C05F0917D05BA
:10410E000E941A23EA0FD001EC93DE011D96EC916A
:10411E00EE0FEE0FEC93FE013D960F01A081E091A4
:10412E007A05F0917B050E941A23EA0FD001EC93D9
:10413E00E0917605EE87E0917C05EF87E0917A05B8
:10414E00E88BA0917E05B0917F05E0914A05F09134
:10415E004B0532960E946C230E2EA0917E05B091D7
:10416E007F051296E0914C05F0914D050E94662355
:10417E000E22A0915E05B0915F05EBEFFFEF0E945E
:10418E005A230E22A0916405B0916505EBEFFFEF67
:10419E000E945A230E22A0910903E0E00E942923D7
:1041AE000E22A0916403E1E00E942923E0211E2E3D
:1041BE00A0916805B0916905E0E0F0E00E9442230D
:1041CE000E2EA0918205B0918305E0E0F0E00E94F2
:1041DE004223E021E12911F40C94F820E0E0E09371
:1041EE006403E8E9E093C1008CE192E00197F1F7F6
:1041FE00E0E0E0936603ABE60E943921E1E0EF8B4D
:10420E00AF89AF3010F00C942521EF89F0E0DE017C
:10421E001296AE0FBF1FEC91A0916603EA0FE093CA
:10422E006603EF89F0E0DE011296AE0FBF1FAC9170
:10423E000E943921EF89EF5FEF8BE2CFA0916603E9
:10424E000E94392184E893E00197F1F714E0E0E948
:10425E00E093C100E0E0E0937903F79A0C940D0A25
:10426E006F96FFCFAA93E091C000E07211F00C940C
:10427E004121F9CFE881E093C6002196089510966A
:10428E0039F088EB9BE00197F1F7A8951197C9F7E4
:10429E000895552342F4503811F4E0FF04C03196CE
:1042AE00691F791F6BF050E8572711F45F93CFC049
:1042BE005F3F31F0660F000C57956795752F089587
:1042CE005F9300200AF0CFC0C8C050E8192E152207
:1042DE00880F991F9527550F879550E8072E0522B1
:1042EE00660F771F7527550F67950895689401C05F
:1042FE00E8945F93F2DF703818F07F3F08F4A7C0A0
:10430E0056E1571BAAF4519558300EF4593030F03F
:10431E00EFEFFFEF6FEF7FE777F91AC0772755239F
:10432E00B9F0EE0FFF1F661F771F5A95D1F710C019
:10433E007727583028F0EF2FF62F672F5850F9CFE8
:10434E00552331F076956795F795E7955A95D1F700
:10435E0000200AF44FD15F910895689401C0E8944B
:10436E00309760407040B1F0002426F0772312F4AD
:10437E00009440D1172E7EE1112032F07A95EE0F87
:10438E00FF1F661F111CF9CFEF2FF62F612D5F93C4
:10439E008ADF5F9108954F93AF01FD01DA01AB0102
:1043AE00BC01CA01402D012C142E4F910895EA0F25
:1043BE00FB1F681F0895E095F0956095EF5FFF4F26
:1043CE006F4F08955F9381DF903871F150E8152695
:1043DE0004C05F937ADF903839F1703821F1572F8E
:1043EE00591B2BF112F4D7DFFACF583118F0AA2748
:1043FE00BB278827583028F0AB2FB82F8827585066
:10440E00F9CF552329F08695B795A7955A95D9F7E3
:10441E00502D512572F0CBDF38F46795F795E7955F
:10442E00739513F420C0B7DF3EDF5F910895D8F780
:10443E00FBCFEA1BFB0B680B51F010F40094BBDFB3
:10444E00662392F3EE0FFF1F661F7A95CBF7EE27CA
:10445E00FF27662777275F910895EFEFFFEF6FE74E
:10446E007FEF5F910895EFEFFFEF6FE77FE75F91CB
:10447E0008955F932ADF703851F3903841F3012489
:10448E000894791F23F41CF300203AF3ECCF0F921B
:10449E001F932F933F934F93112722279927689F9E
:1044AE00A0018F9F302D410D591F6B9F300D411D67
:1044BE00591F8E9F27D0BF9F25D06A9F23D0BE9FA6
:1044CE001DD0AF9F1BD0AE9F110D291F391F491F45
:1044DE00591FE32FF42F652F522F4F913F912F919C
:1044EE001F910F9066232AF0550FEE1FFF1F661FB8
:1044FE0002C073954BF2CDDE5F910895100D211D14
:10450E00391F02C0200D311D491F591F08955F9399
:10451E00DCDE703821F411200AF49FCFA4CF90383E
:10452E0009F495CF01240894970B1BF4D4F30020C3
:10453E00F3CF792F1F932F933F934F93112411276E
:10454E00222733274427552790E2AE17BF07860749
:10455E00410730F0AE1BBF0B860B410B089401C018
:10456E008894551F221F331F111CAA1FBB1F881FA3
:10457E00441F9A9551F7F901612D4F913F912F915B
:10458E001F91662332F0550FEE1FFF1F661F7A959F
:10459E0043F27FDE5F91089599239AF0772342F0DC
:1045AE00971748F029F4AE17BF07860720F031F0B1
:1045BE0098948894089598940894089518948894DB
:1045CE0008957723C2F7971798F3A9F7EA17FB0711
:1045DE00680788F399F3ECCFEA0FFB1F681F791F6A
:1045EE000895EA1BFB0B680B790B0895F195E19585
:1045FE00F0400895F09560957095E195FF4F6F4FDF
:10460E007F4F0895EE230E2EEA2F19F0E6950A94A9
:10461E00E9F70895EE230E2EFD0121F0F595E795AD
:10462E000A94E1F70895EF2FFF27E7FDFFEF0895B6
:10463E006F2F660F660B762F08958B2F880F880BC2
:10464E00982F0895EA17E1E009F0EE270895EA178A
:10465E00E1E009F4EE270895AE17E1E008F4EE2745
:10466E000895AE17E1E008F0EE270895EA17E1E0AD
:10467E0008F0EE270895EA17FB07E1E009F0EE27B0
:10468E000895EA17FB07E1E009F4EE270895EA170B
:10469E00FB07E1E00CF4EE270895AE17BF07E1E04B
:1046AE000CF4EE270895AE17BF07E1E00CF0EE27ED
:1046BE000895EA17FB07E1E00CF0EE270895AE1718
:1046CE00BF07E1E008F0EE270895EA17FB07E1E0E7
:1046DE0008F0EE270895AE17BF0786079707E1E0AB
:1046EE000CF0EE270895EA17FB0768077907E1E05B
:1046FE000CF0EE270895FA9FF02DEB9FF00DEA9F38
:10470E00E02DF10D08957A9F702D6B9F700DF89F1F
:10471E00700DE99F700D6A9F602D710DFB9F600DEE
:10472E00711DE89F600D711D8827FA9FF02D610D98
:10473E00781FEB9FF00D611D781FEA9FE02DF10DA4
:10474E00681F781F08954BD0D6DF0EF44FDF089503
:10475E0054D0D9DF0EF44EDF08950024112490E1D9
:10476E00AA0FBB1F001C111C0E1A1F0A18F40E0EE6
:10477E001F1E01C0A1609A9599F7FD01D001089501
:10478E002ED0EBDF0EF432DF08953F934F935F93FD
:10479E00002411244427552730E2AA0FBB1F881F7F
:1047AE00991F001C111C441F551F0E1A1F0A460B81
:1047BE00570B28F40E0E1F1E461F571F01C0A16077
:1047CE003A9559F7FD01BC01D001CA015F914F9195
:1047DE003F91089512D0D9DF0EF40CDF0895E894BE
:1047EE00F7FF02C003DF6894B7FF06C0A095B0952F
:1047FE00119600F8039400FA0895E89477FF02C02A
:10480E00F9DE689497FF0BC00024A095B0958095B3
:10481E0090951196801D901D00F8039400FA08954E
:10482E00ED93FD936D937C930895182E862F612D35
:10483E00192E972F712D1B2EBF2FF12D1A2EAE2F45
:10484E00E12D0895F999FECFFF93FFB7F894A1BD1E
:10485E00B2BDF89AE0B5FFBFFF910895F99B02C073
:10486E00A895FCCF9FB7F894A1BDB2BDF89A80B5BC
:10487E00E81719F0E0BDFA9AF99A9FBF089500243F
:10488E000A160B06089500240A160B0608060906DA
:10489E000895AC0FBD1F05900D928A95E1F708950E
:00000001FF
